:100000000C942A000C9447000C9447000C94470071
:100010000C9447000C9447000C9449000C94470042
:100020000C9447000C9447000C9447000C94470034
:100030000C9447000C9447000C9447000C94470024
:100040000C9447000C9447000C9447000C94470014
:100050000C94470011241FBECFE5D4E0DEBFCDBF16
:1000600010E0A0E6B0E0E0EEF0E002C005900D92F6
:10007000A036B107D9F710E0A0E6B0E001C01D92AC
:10008000A136B107E1F70E9463000C946F000C9455
:1000900000001F920F920FB60F9211248F93809140
:1000A00060008F5F8093600080916000883228F04C
:1000B0008BB380958BBB109260008F910F900FBE19
:1000C0000F901F9018958FEF8ABB8DE08EBD8DE04D
:1000D00091E09BBD8ABD80E189BF7894FFCFFFCFBF
:00000001FF
